:04FFF00023001E00CC
:08FFF800000000000000000001
:03000000022F6765
:0C2F670078FFE4F6D8FD75817E022FAEE5
:10362D0057502053657175656E63657200302E3687
:0D363D00004D6179203330203230303600EE
:023386008F2690
:10338800E4F527F528C3E5289526E527940050237A
:10339800900000AF82AE83E4FCFD7B107A27F9F839
:1033A800D312131E4003A380EA0528E52870D6052A
:0333B8002780D299
:0133BB0022EF
:1034A0007BFF7A36792D1236B912374C7F76123778
:1034B000727BFF7A36793A1236B912374C7BFF7A33
:0934C00036793E1236B902374C90
:102CE7001236F112372F12367BE4F524E4F5257DF1
:102CF70001AF251234F07F01123386E4FDAF2512B0
:102D070034F00525E525C3940340E40524E524C3F1
:102D1700940540D812376F7B017A01799A7536008E
:102D270075370CE4FFFE1232C290019AE064AB7073
:102D370004A3E064CD603912376090019A74ABF058
:102D4700A374CDF0A37401F0E4A3F0A3F0A31213CE
:102D5700AB3D4CCCCDE49001A3F0A304F0E4A3F089
:102D67007B017A01799AF53675370CFFFE12330429
:102D770090019CE0D39405400374C0F0C390019E7A
:102D8700E0943C90019DE094004006E4F0A3743B7E
:102D9700F020970B7D017F01123073D2AF80FE9038
:102DA700019CE0FDE4FF123073D2AF1234A0E4F5CA
:102DB7000E1235CBD20EA296920BA297920C12331B
:102DC70046E50E60FCE4F50E12146712369180F1A9
:03376F00C216225D
:10356000AD07AC062016FDD216EC5401F5F1EDF5D1
:10357000F330AF0320EF0AE5F130E7FBC216AFF2FC
:04358000227F002284
:04344A00AB07AA061C
:10344E002016FDD216EA5401F5F1A2AF9200C2AFDA
:10345E008DF2EBF5F3A20092AF30AF0320EF07E54C
:06346E00F130E7FBC2167D
:013474002235
:0433F000AB07AA0677
:1033F4002016FDD216EA54014420F5F1A2AF92152D
:10340400C2AF8DF2EBF5F3A21592AF30AF0320EF0C
:0834140007E5F130E7FBC216E9
:01341C00228D
:103516002016FDD21675F131A2AF9200C2AF8FF21E
:10352600E4F5F3A20092AF30AF0320EF07E5F130E8
:04353600E7FBC216D7
:01353A00226E
:05375B00E4FD0233F063
:05376000E4FF02351634
:03007300023755FC
:0637550053F17FC21632A1
:0A32C2008E318F328B338A34893548
:1032CC00E4F538F539C3E5399537E53895365027A7
:1032DC00E5322539FFE5313538FE123560AB33AABE
:1032EC0034A935853982853883EF1211B20539E559
:0732FC003970D2053880CEC5
:0133030022A7
:0A3304008E318F328B338A34893505
:10330E00E4F538F539C3E5399537E5389536502764
:10331E00E5322539FFE5313538FEAB33AA34A93510
:10332E00853982853883121173FD12344A0539E5C9
:07333E003970D2053880CE82
:013345002265
:10316600256C660025303264253032642E253034D5
:10317600642C25630025303364253032642E2530D7
:1031860034642C256300252E33660025332E3266E3
:1031960000244750524D422C412C302C4C2C2530CB
:1031A60033642C253033642C002C002C3030302E28
:0E31B600302C00573A002C523A002C423A00BE
:0437650041012600F8
:0A35A800E0FF7E007B017A0079ABA2
:1035B200EF7803C333CE33CED8F92420FFE43EFEA6
:0935C2007536007537080232C2AB
:10364A00EF7803C333CE33CED8F92420FFE43EFE0D
:09365A00753600753708023304CF
:1031C4002094028028900125E004F0E0FF90019D06
:1031D400E0FCA3E0FDD39FEC940050359001A4E003
:1031E400601E24FE60248000900125EDF078AB7C05
:1031F400007D017B017A0179277E007F080211346A
:1032040090019DA3E0900125F022E4900125F08037
:08321400039001251235A822E8
:102FF300E4F531F532E53225E02457F8E4F608F636
:103003000532E532700205316414453170E7E4F5A9
:1030130031F53212115AFF600CB42009740129F9F9
:10302300E43AFA80EEEF6043AE02AF010532E532D7
:10303300700205311425E02457F8A60608A60712E6
:10304300115AFF600D642C6009740129F9E43AFAFE
:1030530080EDEF600CE41211A00429F9E43AFA8040
:0F306300028008E5326414453170A8AE31AF32F7
:01307200223B
:10254000753AFF753B31753C66753D01753E017509
:102550003F4712226FE4FBFA79C87842900147E0C6
:10256000FCA3E0FDA3E0FEA3E0FF120C9B120DF420
:1025700090014FEEF0A3EFF0900147E0FCA3E0FDE7
:10258000A3E0FEA3E0FFC004C005C006C0079001A1
:102590004FE0FCA3E0FDE4120DBBE4FBFA79C87840
:1025A00042120B92A804A905AA06AB07D007D006D1
:1025B000D005D004120A9D90014712139F90014745
:1025C000E0FCA3E0FDA3E0FEA3E0FF120DF4900108
:1025D00051EEF0A3EFF0900147E0FCA3E0FDA3E093
:1025E000FEA3E0FFC004C005C006C007900151E093
:1025F000FCA3E0FDE4120DBBA804A905AA06AB07E5
:10260000D007D006D005D004120A9D9001471213BE
:102610009F900147E0FCA3E0FDA3E0FEA3E0FFE400
:10262000FBFA79707842120B9290014712139F9037
:102630000151E0FCA3E0FDE4120DBBE4FBFA79706C
:102640007842120C9BC004C005C006C00790014F21
:10265000E0FCA3E0FDE4120DBBD003D002D001D01A
:1026600000120AA1C004C005C006C007E4FBFA7945
:10267000617845900147E0FCA3E0FDA3E0FEA3E004
:10268000FF120C9BD003D002D001D000120AA190FF
:10269000014B12139FAB34AA35A93612115AFF64AD
:1026A000576004EFB4531790014BE0FCA3E0FDA387
:1026B000E0FEA3E0FF120DA590014B12139F9001C5
:0C26C0004BE0FCA3E0FDA3E0FEA3E0FF64
:0126CC0022EB
:10358400753AFF753B31753C66753D01753E0175B5
:103594003F3612226F900136E0FCA3E0FDA3E0FE6B
:0335A400A3E0FFA2
:0135A7002201
:082AA7008F348E338D328C3127
:102AAF00123722120DF4900147EEF0A3EFF0AF347E
:102ABF00AE33AD32AC31123722C004C005C006C0F0
:102ACF0007900147E0FCA3E0FDE4120DBBA804A9A9
:102ADF0005AA06AB07D007D006D005D004120A9D71
:102AEF00E4FBFA79707842120B9290014D12139F0A
:102AFF0090014DE0FCA3E0FDA3E0FEA3E0FF120D6B
:102B0F00F4900149EEF0A3EFF090014DE0FCA3E04B
:102B1F00FDA3E0FEA3E0FFC004C005C006C0079000
:102B2F000149E0FCA3E0FDE4120DBBA804A905AA2E
:102B3F0006AB07D007D006D005D004120A9D90012E
:102B4F004D12139F7F007E407D1C7C4690014DE00F
:102B5F00F8A3E0F9A3E0FAA3E0FB120B92120DF435
:102B6F0090014BEEF0A3EFF07538FF753931753AE0
:102B7F006A900147E0FEA3E08E3BF53CA3E0FEA385
:102B8F00E08E3DF53EA3E0FEA3E08E3FF540E4FF6F
:102B9F00FEFDFCAB34AA33A932A831120D38500414
:102BAF007F5380027F4E8F417B017A0079BC121ACE
:072BBF00187B017A0079BCCC
:012BC60022EC
:082BC7008F348E338D328C3106
:102BCF00123722120DF4900147EEF0A3EFF0AF345D
:102BDF00AE33AD32AC31123722C004C005C006C0CF
:102BEF0007900147E0FCA3E0FDE4120DBBA804A988
:102BFF0005AA06AB07D007D006D005D004120A9D50
:102C0F00E4FBFA79707842120B9290014D12139FE8
:102C1F0090014DE0FCA3E0FDA3E0FEA3E0FF120D49
:102C2F00F4900149EEF0A3EFF090014DE0FCA3E02A
:102C3F00FDA3E0FEA3E0FFC004C005C006C00790DF
:102C4F000149E0FCA3E0FDE4120DBBA804A905AA0D
:102C5F0006AB07D007D006D005D004120A9D90010D
:102C6F004D12139F7F007E407D1C7C4690014DE0EE
:102C7F00F8A3E0F9A3E0FAA3E0FB120B92120DF414
:102C8F0090014BEEF0A3EFF07538FF753931753ABF
:102C9F007B900147E0FEA3E08E3BF53CA3E0FEA353
:102CAF00E08E3DF53EA3E0FEA3E08E3FF540E4FF4E
:102CBF00FEFDFCAB34AA33A932A831120D385004F3
:102CCF007F5780027F458F417B017A0079BC121AB2
:072CDF00187B017A0079BCAB
:012CE60022CB
:103475007538FF753931753A8CE4FBFA797A7844F9
:10348500120C9B8F3E8E3D8D3C8C3B7B017A0079E7
:0B349500BC121A187B017A0079BC22DF
:1035EE007538FF753931753A918F3E8E3D8D3C8C15
:1035FE003B7B017A0079BC121A187B017A0079BCE8
:01360E002299
:10334600C210E49000B7F0900125F01235A8E4FF12
:10335600FE7D207C4190019FE0F8A3E0F9A3E0FA0E
:10336600A3E0FB120B929000B812139FE490011C8D
:10337600F0C211A294B3920FA297B3920C02002648
:10146700A20C309701B3500AA297920C209703124F
:1014770031C4123713EF70030219BB12360F8F26D0
:101487009001A5E06003200E05AF26123772E5260E
:1014970024F8602C24FE604524E6600C24036003D6
:1014A700021995C20E02198DE4900126F0E0FF049F
:1014B700F074CC2FF582E43400F583E526F080B292
:1014C700900126E0D394004003E014F07F08123423
:1014D700C97F201234C97F081234C980959001262C
:1014E700E024CCF582E43400F583E4F0200E0ED23C
:1014F7000E7B017A0079CC121E2B02198D7B017AA3
:101507000079CE900133EBF0A3EAF0A3E9F01213D0
:101517004590012F12139F7F437E4D7D527C509043
:10152700012FE0F8A3E0F9A3E0FAA3E0FBC312134D
:1015370034600302198D7B017A0079CC122FF38571
:101547005C82855B83E064416003021980AA5DA920
:101557005EC0038B34855F35856036D00312254026
:101567009000A312139FAA61A9627B01C0038B3469
:10157700856335856436D0031225409000A7121382
:101587009FAA67A9687B0112358490012112139FD6
:1015970020103B9000B7E004F0E0C3940A402FD23C
:1015A700109000A3E0FCA3E0FDA3E0FEA3E0FF9002
:1015B700012712139F9000A7E0FCA3E0FDA3E0FE24
:1015C700A3E0FF90012B12139F7F031236DF9000D9
:1015D700A7E0FCA3E0FDA3E0FEA3E0F5358E348D84
:1015E700338C32A3E0FCA3E0FDA3E0FEA3E0F539D2
:1015F7008E388D378C36A3E0FCA3E0FDA3E0FEA375
:10160700E0F53D8E3C8D3B8C3A753E01753F00758C
:1016170040B375410175420175431D9000A3E0FC7D
:10162700A3E0FDA3E0FEA3E0FF120076900125E012
:10163700FFD394004006EF14F52D80028F2D7538E7
:10164700FF753931753A97852D3B900125E0753C3B
:1016570000F53D7B017A0079CC121A189000ABE0B7
:10166700FCA3E0FDA3E0FEA3E0FF122AA78B318ACB
:101677003289337B017A0079CC12321C7531FF75C0
:1016870032317533AF7B017A0079CC12321C90006E
:10169700AFE0FCA3E0FDA3E0FEA3E0FF122BC78BA6
:1016A700318A3289337B017A0079CC12321C753149
:1016B700FF7532317533AF7B017A0079CC12321C5A
:1016C7009000B3E0FCA3E0FDA3E0FEA3E0FF12342B
:1016D700758B318A3289337B017A0079CC12321CBF
:1016E7007531FF7532317533AF7B017A0079CC12D2
:1016F700321C90011DE0FCA3E0FDA3E0FEA3E0FF88
:101707001235EE8B318A3289337B017A0079CC121C
:10171700321C7531FF7532317533B17B017A00792F
:10172700CC12321CA20F309401B35006209403123E
:1017370031C4A294920F752756E4F5289001A3E0CF
:10174700703CE4FFFE7D7A7C4490019FE0F8A3E0C3
:10175700F9A3E0FAA3E0FB120B929000B3E0F8A321
:10176700E0F9A3E0FAA3E0FB120D38400302182DBD
:101777007F031236DF7527411231C402182D30114D
:10178700789000B8E0FCA3E0FDA3E0FEA3E0FF90A3
:1017970000B3E0F8A3E0F9A3E0FAA3E0FB120D38E9
:1017A700600A400890011CE004F08005E490011CE9
:1017B700F090011CE0D3940340297F031236DF75B4
:1017C70027411231C4E4FFFE7D207C4190019FE058
:1017D700F8A3E0F9A3E0FAA3E0FB120B929000B89C
:1017E70012139F9000B3E0FCA3E0FDA3E0FEA3E08B
:1017F700FF9000B812139F802DE4FFFE7D7A7C4492
:1018070090019FE0F8A3E0F9A3E0FAA3E0FB120B35
:10181700929000B3E0F8A3E0F9A3E0FAA3E0FB128B
:101827000D385002D2117531007532007533277BA0
:10183700017A0079CC12321CE4F52CF52A752B01BC
:101847007B017A0079CC12000EC3E52B9FEE6480F2
:10185700F8E52A648098501974CC252BF58274001A
:10186700352AF583E0622C052BE52B70D3052A80FA
:10187700CF9001A5E070157B017A0079CC1236B9BB
:101887007F2A123772AF2C12366380647BFF7A315E
:1018970079B91236B9E52D04FF1236637F2C12375A
:1018A70072900125E004FF1236637BFF7A3179BC21
:1018B7001236B99000B3E0FCA3E0FDA3E0FEA3E07D
:1018C700FF120DF47B007A00790012283B7BFF7A28
:1018D7003179C01236B990011DE0FCA3E0FDA3E009
:1018E700FEA3E0FF120DF47B007A00790012283B7B
:1018F70012374C900121E0F8A3E0F9A3E0FAA3E046
:10190700FB90011DE0FCA3E0FDA3E0FEA3E0FF12B6
:101917000A9D120DF48E2A8F2BD3E52B94B4E52A5A
:1019270064809480400C7498252BF52B74FE352A1F
:10193700F52AC3E52B944CE52A6480947F500C74F8
:1019470068252BF52B7401352AF52AC3E52B940559
:10195700E52A6480948050047D01801FD3E52B9491
:1019670005E52A648094804004E4FD80027D017FC0
:10197700011234F07D01E48009E4FD7F011234F0A7
:10198700E4FDFF1234F0E4900126F002147990018F
:1019970026E0FF04F074CC2FF582E43400F583E5EC
:1019A70026F0900126E0C394505003021479E01406
:0419B700F0021479AD
:0119BB002209
:1036F100E4F5847585FF53912FF592F5A475A5FF27
:0137010022A5
:10367B00C214E4FDFF1234F0E4FD7F011234F0E4D8
:06368B00FD7F020234F095
:1034F000EF1460101460162402701ABD0103C2A7F5
:1035000022D2A722BD0103C2A622D2A622BD010358
:06351000D28022C28022DD
:1036DF00EF24FD700CD214750DFA7D017F021234A8
:0236EF00F022C7
:10369100E50DD39400400CD50D09C214E4FD7F0261
:0436A1001234F022CD
:1033BC0025640020200053657474696E67733A00AD
:1033CC0041727269766552616E67653D00206D00D1
:1033DC005365714D6F64653D004379636C654D6F4A
:0433EC0064653D00D7
:061E2B008B2E8A2F893086
:101E310012353BAB2EAA2FA93012115A900136F060
:101E4100121405206B411E7942200243211F441EBA
:101E510076451F434C201A4E21E75020B7511E7280
:101E610052214D53211C561EAD5720E2590000212D
:101E7100F043A20822023760AB2EE5302402F9E4D8
:101E8100352FFA753AFF753B33753CBC753D0175CD
:101E91003E01753F4512226F900145A3E090019CE0
:101EA100F0D39405400374C0F002205BAB2EE53003
:101EB1002402F9E4352FFA122FF3AA57A9587B010E
:101EC100C003753AFF753B33753CBC8B3D753E01D4
:101ED100753F45D00312226FAA59A95A7B01C0034D
:101EE1008B34855B35855C36D00312254090013BF0
:101EF10012139FAA5DA95E7B01C0038B34855F35F8
:101F0100856036D00312254090013F12139F900146
:101F110045E0FEA3E0FFD39400EE6480948050037B
:101F21000221F0D3EF943CEE6480948040030221BF
:101F3100F0EF24FFFFEE34FFFE7B017A01793B02D3
:101F4100364AE4900143F0A3F090019DE0FEA3E046
:101F5100FF900143E0FCA3E0FDC39FEC9E40030220
:101F610021F0C3ED943CEC6480948040030221F0A5
:101F7100900143E0FEA3E0FF7B017A01793B12353A
:101F8100B2900144E02401FF900143E03400FE33AC
:101F910095E0FDFC7B007A00790012283B7BFF7AFB
:101FA1003379BF1236B990013BE0FCA3E0FDA3E019
:101FB100FEA3E0FF122AA7900138EBF0A3EAF0A3F9
:101FC100E9F01236B97BFF7A3379BF1236B9900145
:101FD1003FE0FCA3E0FDA3E0FEA3E0FF122BC790CE
:101FE1000138EBF0A3EAF0A3E9F01236B912374C4D
:101FF100900144E004F07006900143E004F0021FF8
:102001004A123760E490019DF0A3F07B017A0179D7
:102011009AF53675370C022148AB2EE5302402F9CA
:10202100E4352FFA753AFF753B33753CBC753D01BC
:10203100753E01753F4512226F900145E0FEA3E018
:10204100FF90019DEEF0A3EFF0C3943CEE940040AD
:102051000990019DE4F0A3743BF07B017A01799A28
:1020610075360075370CE4022148AB2EE5302402A9
:10207100F9E4352FFA753AFF753B33753CBC753D74
:1020810001753E01753F4512226F900145E0FCA3A9
:10209100E0FDEC120DBBE4FBFA797A7844120C9B5B
:1020A10090019F12139F7B017A01799A7536007511
:1020B100370CE4022148AB2EAA2FA930900002125E
:1020C1001173B444089001A37401F08005E49001F8
:1020D100A3F07B017A01799A75360075370CE4809B
:1020E10066AB2EAA2FA93090000212117324CF6083
:1020F1000E24DF601180009001A47401F0800DE4D2
:102101009001A4F080069001A47402F07B017A0191
:10211100799A75360075370CE4802C0234A0AB2E09
:10212100AA2FA930900002121173B431089001A5B1
:102131007401F08005E49001A5F07B017A01799AA0
:1021410075360075370CE4FFFE0233047BFF7A33EA
:1021510079C21236B912374C7BFF7A3379CC1236F9
:10216100B9E4FFFE7D7A7C4490019FE0F8A3E0F999
:10217100A3E0FAA3E0FB120B92120DF47B007A00AC
:10218100790012283B7BFF7A3379D91236B912379D
:102191004C7BFF7A3379DC1236B99001A3E07004ED
:1021A1007F4180027F4412377212374C7BFF7A33B2
:1021B10079E51236B99001A4E0600F24FE601304A2
:1021C10070169001377448F0800E9001377431F029
:1021D10080069001377452F0900137E0FF12377298
:0F21E10012374C02374C7D017F0112307380FEA4
:0121F00022CC
:10002600E4F529F528F527F526AB29AA28A927A856
:1000360026AF29AE28AD27AC26120A9DC004C005FE
:10004600C006C007AB29AA28A927A826AF29AE282B
:10005600AD27AC26120A9DD003D002D001D00012E3
:0A0066000C9B8F0B8E0A8D098C088D
:01007000226D
:080076008F318E308D2F8C2E8E
:10007E009001361213AB3B5CA8F190013A1213AB10
:10008E004AC2A72890013E1213AB29612E1390018C
:10009E00421213AB42652EE0900136E0F8A3E0F970
:1000AE00A3E0FAA3E0FBE4FFFE7D807C3F120A9DF5
:1000BE0090014612139F900142E0F8A3E0F9A3E0ED
:1000CE00FAA3E0FBAF31AE30AD2FAC2E120C9B126B
:1000DE00275D900146E0F8A3E0F9A3E0FAA3E0FB68
:1000EE00120B9290014A12139F900142E0F8A3E086
:1000FE00F9A3E0FAA3E0FBAF39AE38AD37AC361258
:10010E000C9B12275D900146E0F8A3E0F9A3E0FAFC
:10011E00A3E0FB120B9290014E12139F90014AE046
:10012E00FCA3E0FDA3E0FEA3E0FFA804A905AA0638
:10013E00FB120B92E4FBFA7980783F120AA1122E81
:10014E00C1A804A905AA06AB07E4FFFE7D807C3F8B
:10015E00120C9B90015212139F90014AE0FCA3E0F7
:10016E00FDA3E0FEA3E0FF900152E0F8A3E0F9A3A7
:10017E00E0FAA3E0FB120B9290015612139F90012E
:10018E004EE0FCA3E0FDA3E0FEA3E0FFA804A9055A
:10019E00AA06FB120B92E4FBFA7980783F120AA1B1
:1001AE00122EC1A804A905AA06AB07E4FFFE7D80A6
:1001BE007C3F120C9B90015A12139F90015AE0FC47
:1001CE00A3E0FDA3E0FEA3E0FF900152E0F8A3E060
:1001DE00F9A3E0FAA3E0FB120B9290015E12139FBB
:1001EE0090014EE0FCA3E0FDA3E0FEA3E0FF900132
:1001FE005EE0F8A3E0F9A3E0FAA3E0FB120B929005
:10020E00016212139F90014AE0FCA3E0FDA3E0FE01
:10021E00A3E0FF900162E0F8A3E0F9A3E0FAA3E007
:10022E00FB120B9290016612139FAB35AA34A933C1
:10023E00A832AF3DAE3CAD3BAC3A120A9D900142A6
:10024E00E0F8A3E0F9A3E0FAA3E0FB120C9B900107
:10025E006A12139F90016AE0FCA3E0FDA3E0FEA3E7
:10026E00E0FF12272B90017212139F90016AE0FC9F
:10027E00A3E0FDA3E0FEA3E0FF1227159001761286
:10028E00139F900172E0FCA3E0FDA3E0FEA3E0FF4C
:10029E0090015AE0F8A3E0F9A3E0FAA3E0FB120BF9
:1002AE009290014A12139F90015AE0FCA3E0FDA325
:1002BE00E0FEA3E0FF900156E0F8A3E0F9A3E0FA18
:1002CE00A3E0FB120B92900176E0F8A3E0F9A3E015
:1002DE00FAA3E0FB120B92A804A905AA06AB07909D
:1002EE000162E0FCA3E0FDA3E0FEA3E0FF120A9D85
:1002FE0090014E12139F90014EE0FCA3E0FDA3E08F
:10030E00FEA3E0FFA804A905AA06FB120B92C004E7
:10031E00C005C006C00790014AE0FCA3E0FDA3E0C3
:10032E00FEA3E0FFA804A905AA06FB120B92D003B8
:10033E00D002D001D000120AA1122EC190017A1261
:10034E00139F900176E0FCA3E0FDA3E0FEA3E0FF87
:10035E0090015EE0F8A3E0F9A3E0FAA3E0FB120B34
:10036E0092900166E0F8A3E0F9A3E0FAA3E0FB1295
:10037E000AA190017E12139F90017EE0FCA3E0FD86
:10038E00A3E0FEA3E0F54B8E4A8D498C4890017A8E
:10039E00E0FCA3E0FDA3E0FEA3E0FF1230F390012A
:1003AE009212139F900172E0FCA3E0FDA3E0FEA366
:1003BE00E0FF90015EE0F8A3E0F9A3E0FAA3E0FB12
:1003CE00120B9290017AE0F8A3E0F9A3E0FAA3E011
:1003DE00FB120C9B90019612139F900196E0FCA3CA
:1003EE00E0FDA3E0FEA3E0FF120DA5900196E0F85C
:1003FE00A3E0F9A3E0FAA3E0FB120B92E4FBFA7977
:10040E0080783F120AA190018612139F900166E038
:10041E00FCA3E0FDA3E0FEA3E0FFA804A905AA0645
:10042E00FB120AA190018212139FE4FFFEFDFC90C5
:10043E000186E0F8A3E0F9A3E0FAA3E0FB120D3881
:10044E00603B4039900182E0FCA3E0FDA3E0FEA3F7
:10045E00E0FF120DA5900186E0F8A3E0F9A3E0FA03
:10046E00A3E0FB120C9B90017EE0F8A3E0F9A3E061
:10047E00FAA3E0FB120AA190018212139F9001824F
:10048E00E0FCA3E0FDA3E0FEA3E0FFA804A905AAFB
:10049E0006FB120B92E4FBFAF97840120B92E4FB86
:1004AE00FA798078BF120AA190018E12139FE4FF91
:1004BE00FE7D407CC0900186E0F8A3E0F9A3E0FA4F
:1004CE00A3E0FB120B92E4FBFA79807840120AA1AA
:1004DE00900136E0F8A3E0F9A3E0FAA3E0FB120BDB
:1004EE0092E4FBFA79807840120AA1900186E0F836
:1004FE00A3E0F9A3E0FAA3E0FB120B92900136E021
:10050E00F8A3E0F9A3E0FAA3E0FB120B92E4FBFAE6
:10051E0079807841120C9B90018A12139F90016A88
:10052E00E0FCA3E0FDA3E0FEA3E0FFA312139F9067
:10053E00017EE0FCA3E0FDA3E0FEA3E0FF90018EB0
:10054E00E0F8A3E0F9A3E0FAA3E0FB120B9290010E
:10055E008AE0F8A3E0F9A3E0FAA3E0FB120B929075
:10056E000182E0F8A3E0F9A3E0FAA3E0FB120AA1EE
:10057E0090017AE0F8A3E0F9A3E0FAA3E0FB120BF6
:10058E009290018AE0F8A3E0F9A3E0FAA3E0FB124F
:10059E000B92900192E0F8A3E0F9A3E0FAA3E0FB3E
:1005AE00120AA1900196E0F8A3E0F9A3E0FAA3E005
:1005BE00FB120B9290016A12139F90018AE0F8A32E
:1005CE00E0F9A3E0FAA3E0FBE4FFFE7D807C3F129E
:1005DE000A9D90016AE0F8A3E0F9A3E0FAA3E0FB1C
:1005EE00120B92900136E0F8A3E0F9A3E0FAA3E033
:1005FE00FB120B92C004C005C006C007AB35AA346F
:10060E00A933A832AF3DAE3CAD3BAC3A120A9D9039
:10061E000142E0F8A3E0F9A3E0FAA3E0FB120C9B81
:10062E00D003D002D001D000120AA190016A121399
:10063E009F90016AE0F8A3E0F9A3E0FAA3E0FBA320
:10064E00E0FCA3E0FDA3E0FEA3E0FF120A9D12373B
:10065E002290013EE0F8A3E0F9A3E0FAA3E0FB123A
:10066E000D38500302026290014EE0FCA3E0FDA3A0
:10067E00E0FEA3E0F54B8E4A8D498C4890014AE08E
:10068E00FCA3E0FDA3E0FEA3E0FF1230F3900166B1
:10069E0012139F900172E0FCA3E0FDA3E0FEA3E025
:1006AE00FF900152E0F8A3E0F9A3E0FAA3E0FB12F9
:1006BE000B92C004C005C006C00790015AE0FCA30F
:1006CE00E0FDA3E0FEA3E0FF900156E0F8A3E0F901
:1006DE00A3E0FAA3E0FB120B92C004C005C006C053
:1006EE0007900176E0FCA3E0FDA3E0FEA3E0FF90FF
:1006FE000162E0F8A3E0F9A3E0FAA3E0FB120B928B
:10070E00D003D002D001D000120A9D8F4B8E4A8D9D
:10071E00498C48D007D006D005D0041230F37BDBCD
:10072E007A0F79497840120AA190016212139F90B4
:10073E000146E0F8A3E0F9A3E0FAA3E0FBE4FFFE34
:10074E007D807C3F120C9B900146E0F8A3E0F9A35C
:10075E00E0FAA3E0FB120C9BE4FBFA798078BF125F
:10076E000AA1900186E0F8A3E0F9A3E0FAA3E0FB6A
:10077E00120B92E4FBFA7980783F120AA1122EC175
:10078E00E4FBFA7980783F120AA190016A12139F56
:10079E00E4FFFEFD7CC090016AE0F8A3E0F9A3E05F
:1007AE00FAA3E0FB120AA190016AE0F8A3E0F9A314
:1007BE00E0FAA3E0FB120C9B90016A12139F9001CA
:1007CE006AE0F8A3E0F9A3E0FAA3E0FBE4FFFE7D04
:1007DE00807C3F120A9D90018A12139F90016AE05D
:1007EE00FCA3E0FDA3E0FEA3E0FF90016AE0F8A306
:1007FE00E0F9A3E0FAA3E0FB120B92E4FBFA798096
:10080E007840120C9BE4FBFA7980783F120AA19093
:10081E00018AE0F8A3E0F9A3E0FAA3E0FB120C9B37
:10082E0090018A12139FE4FFFE7DC07C3E90016A08
:10083E00E0F8A3E0F9A3E0FAA3E0FB120B9290011B
:10084E006AE0F8A3E0F9A3E0FAA3E0FB120B92E44E
:10085E00FBFA798078BF120AA190016AE0F8A3E052
:10086E00F9A3E0FAA3E0FB120B9290016E12139F14
:10087E0090017EE0FCA3E0FDA3E0FEA3E0FF90016B
:10088E008EE0F8A3E0F9A3E0FAA3E0FB120B92903E
:10089E00016A12139F90018EE0FCA3E0FDA3E0FE1F
:1008AE00A3E0FF90018EE0F8A3E0F9A3E0FAA3E045
:1008BE00FB120B92A804A905AA06AB07E4FFFE7D66
:1008CE00807C3F120A9D90015E12139F90017AE088
:1008DE00FCA3E0FDA3E0FEA3E0FFA804A905AA0681
:1008EE00FB120B92E4FBFA79807840120B92E4FB38
:1008FE00FA794078C0120AA190015EE0F8A3E0F9FF
:10090E00A3E0FAA3E0FB120B92900182E0F8A3E0C1
:10091E00F9A3E0FAA3E0FB120B9290016EE0F8A3AC
:10092E00E0F9A3E0FAA3E0FB120B92E4FBFA79C024
:10093E007840120C9B90016AE0F8A3E0F9A3E0FA6C
:10094E00A3E0FB120A9D90016EE0F8A3E0F9A3E08C
:10095E00FAA3E0FB120B92E4FBFA79807840120CBA
:10096E009B900182E0F8A3E0F9A3E0FAA3E0FB126A
:10097E000AA190017AE0F8A3E0F9A3E0FAA3E0FB64
:10098E00120B9290016EE0F8A3E0F9A3E0FAA3E057
:10099E00FB120B92900192E0F8A3E0F9A3E0FAA308
:1009AE00E0FB120AA190018AE0F8A3E0F9A3E0FAB5
:1009BE00A3E0FB120B9290013AE0F8A3E0F9A3E05A
:1009CE00FAA3E0FB120B92900146E0F8A3E0F9A324
:1009DE00E0FAA3E0FB120B9290015E12139F9001BE
:1009EE005EE0FCA3E0FDA3E0FEA3E0FFAB3EAA3F6A
:1009FE00A940121365900142E0FCA3E0FDA3E0FEC6
:100A0E00A3E0FF900166E0F8A3E0F9A3E0FAA3E00B
:100A1E00FB120B92AB41AA42A943121365AB41AA3A
:100A2E0042A943121345E4FBFA79B47843120D3808
:100A3E005022AB41AA42A943C003C002C001121307
:100A4E0045E4FBFA79B47843120A9DD001D002D066
:100A5E0003121365AB41AA42A943121345E4FBFAF4
:100A6E00F9F8120D3860244022AB41AA42A943C0C6
:100A7E0003C002C001121345E4FBFA79B4784312A5
:0B0A8E000AA1D001D002D003121365B2
:010A9900223A
:0A372F00E4F5955396BF53A27F22E4
:1035CB005389F0438901538FFE758C70E4F58A5350
:1035DB00B8FD53B7FDD2A9D28C53890F43899053B1
:0335EB008FEF223D
:03000B0002374376
:09374300050E758C70758A0032C8
:1036A5000D0A00303132333435363738394142432B
:0436B5004445460042
:103073005387BF75985053877FE4F5BABF01054363
:10308300A240800353A2BFE4F5BDED1460151460A4
:103093001A14601F1460242404702575BEF075BFD4
:1030A3000B802375BEF075BF05801B75BEF075BF21
:1030B30002801375BE7075BF01800B75BEB08003AF
:1030C30075BE30E4F5BF75BD035391FE43920143D2
:1030D30091025392FDC21753B8EF53B7EF43B810A1
:1030E300E49000A1F09000A0F09000A2F0D2AC22F6
:0300230002327432
:10327400C0E0C083C082C0D075D0103098309000B8
:10328400A1E0C3949F50259000A0E0FF04F07400D7
:103294002FF582E43400F583E599F09000A1E00471
:1032A400F09000A0E0C394A04002E4F0C2983099EA
:0E32B40004C299C217D0D0D082D083D0E032AD
:080003002017FDD2178F99228E
:10341D009000A1E0D394004021A3E0FF04F07400DC
:10342D002FF582E43400F583E0FF9000A1E014F065
:0C343D00A3E0C394A04005E4F0227F004F
:013449002260
:033772000200034F
:10360F007F207E4E9000A1E07010D3EF9400EE94D7
:0D361F00004007EF1F70ED1E80EA12341D01
:01362C00227B
:1036B90012115AFF600C123772740129F9E43AFAAF
:0336C90080EE226E
:0F3713009000A1E0D3940040037F01227F0022A9
:10366300AE07EE54F0C4540F9036A893FF1237728E
:08367300EE540F93FF023772C1
:09374C007BFF7A3679A50236B93B
:10353B0012115AFF601EC3648094E1400ED3EF64F6
:10354B008094FA5006EF24E01211A0740129F9E4DB
:04355B003AFA80DCDC
:01355F002249
:0E283B008F348E338D328C318B358A3689374F
:10284900E4F541EC4D4E4F701EE94A4B70057F305F
:10285900023772AB35AA36A937AF4105418F827568
:102869008300743002297BAE33AD32AC31EC335086
:1028790036E5374536453570077F2D123772801496
:10288900AB35AA36A937AF4105418F8275830074EC
:102899002D1211B2AF34AE33AD32AC311213108FE9
:1028A900348E338D328C31754001753B00753ACACF
:1028B90075399A75383BE4FFFEFDFCAB3BAA3AA992
:1028C90039A838D31213345003022966AF34AE3312
:1028D900AD32AC31A83812127E8F3F8E3E8D3D8CC1
:1028E9003CEC4D4E4F7004E5407028E53F2430FF25
:1028F900E5374536453570051237728013AB35AA71
:1029090036A937AE4105418E82758300EF1211B2A7
:10291900E4F540AF3BAE3AAD39AC38AB3FAA3EA97E
:102929003DA83C1211F3AA06A905A804C3E5349FE2
:10293900F534E5339AF533E53299F532E53198F511
:1029490031AF3BAE3AAD39AC38E47B0AFAF9F8124B
:10295900127E8F3B8E3A8D398C380228BFE5364579
:102969003745356010AB35AA36A93785418275835D
:0529790000E41211B2A0
:01297E002236
:100A9A00020E60E86480F8E933E83360110460F01C
:100AAA00ED33EC337009E8FCE9FDEAFEEBFF2204C2
:100ABA0060DED3EB9FEA9EE99DE8C2E78CF0C2F7BD
:100ACA0095F0400CE8CCF8E9CDF9EACEFAEBCFFB89
:100ADA00120E2B85D0F05804700320D5B3E80470A9
:100AEA00075002B2D5020E6A92D5EC0460F7E4CC44
:100AFA00C0E0C398F8603B94186008400DD0E0FB52
:100B0A00020E42E4FBFAC9FC8028E830E406E4C994
:100B1A00FBE4CAFCE830E305E4C9CACBFCE85407A5
:100B2A006010F8C3E913F9EA13FAEB13FBEC13FCB0
:100B3A00D8F130F52FC3E49CFCEF9BFFEE9AFEED53
:100B4A0099FDD0E0FBEF4E4D4C701222DB03020EF2
:100B5A0067EC2CFCEF33FFEE33FEED33FDED30E7AF
:100B6A00EB020E42EF2BFFEE3AFEED39FDD0E0FB31
:100B7A0050130BBB0003020E6AED13FDEE13FEEFDA
:080B8A0013FFEC13FC020E4204
:100B9200EC4D6011E8497017ED33EC3304600DE45D
:100BA200FCFFFEFD22E933E8330470F8020E601206
:100BB2000E2B58046009E4CC248150062850090207
:100BC2000E6A284003020E67C0E0EB4A7044B98007
:100BD20006D0E0FB020E56EF4E701CBD8008EBFF04
:100BE200EAFEE9FD80EBE98DF0A4FEE5F0020C7B64
:100BF200E9CDF9EAFEEBFFEF89F0A4FCE5F0CE893E
:100C0200F0A42EFFE435F0CD89F0A42DFEE435F0FA
:100C12008067EF4E7005BD80D780C3EF8BF0A4AC28
:100C2200F0EE8BF0A42CFCE435F0F8EF8AF0A42C63
:100C3200E5F038FCE433CB8DF0A42CFCE5F03BF876
:100C4200EE8AF0A42CFCE5F038F8E433CF89F0A466
:100C52002CFCE5F038CF3400CE89F0A42FFFE5F06C
:100C62003EFEE433C98DF0A42EFEE5F039CD8AF0C4
:100C7200A42FFFE5F03EFEE43DFD33D0E0FB50073C
:100C82000BBB000F020E6AEC2CFCEF33FFEE33FEBF
:060C9200ED33FD020E42ED
:100C9800020E6AEC5D046005E859047003020E60F8
:100CA800120E2B580460F6EC4860F2EC7004FDFE5E
:100CB800FF22C860DB2481C85009C398600250062F
:100CC800020E679850CAF582E9294B4A7005AB8233
:100CD800020E5675F0007C1A7880C3EF9BEE9AEDF1
:100CE80099400DC3EF9BFFEE9AFEED99FDE842F0A7
:100CF800DC23ACF0D0E0FFD0E0FED0E0FDAB8220FA
:100D0800E7101BEB60BAEC2CFCEF33FFEE33FEED83
:100D180033FD020E42E803F830E705C0F075F00035
:100D2800EF2FFFEE33FEED33FD40B830E7C280AA67
:100D380074F8CC6480CCC86480C8F582046043C36E
:100D4800EB9FF5F0EA9E42F0E99D42F0E89C45F001
:100D580060305018E5825FFFE582F42B5582FB5026
:100D6800210ABA001D09B90019088016E5825BFB43
:100D7800E582F42F5582FF50090EBE00050DBD0017
:100D8800010CC3EB9FF5F0EA9E42F0E99D42F0E8C2
:0D0D98009C45F06007CC4820E701B3EC2239
:100DA500ED33EC33600A047003BD8004ECB2E7FC5C
:010DB500221B
:100DB60075F020800E75F010800575F0087D007EB8
:100DC600007F003392D530D503121310EC33401058
:100DD600EF33FFEE33FEED33FDEC33FCD5F0ED22C1
:0E0DE600E5F0247EA2D513CC92E7CDCEFF22FD
:100DF400EDD2E7CD33EC3392D524814006E4FFFEF7
:100E0400FDFC22FCE4CFCECDCC24E0501174FF8055
:100E1400EDC3CC13CCCD13CDCE13CECF13CF0470F2
:070E2400F030D5DE021310CF
:1019BC00E54C2438F8E6054C2278353007027838A7
:1019CC00E475F0011213E502115A2000EB7F2ED2C0
:1019DC00008018EF540F2490D43440D4FF30040B03
:1019EC00EF24BFB41A0050032461FFE54D600215CB
:1019FC004D0550E5507002054F30070D7835E475F4
:101A0C00F0011213E5EF0211A00234C97403D207DE
:101A1C008003E4C207F54C8B358A368937E4F54DE3
:101A2C00F54FF550E54D60077F201219F780F575DD
:101A3C004EFFC201C200C202C203C205C206C208E6
:101A4C001219C5FF700D3007057F00121A08AF5030
:101A5C00AE4F22B4255FC2D5C2041219C5FF24D0E3
:101A6C00B40A00501A75F00A784D30D50508B6FF47
:101A7C000106C6A426F620D5047002D20380D92410
:101A8C00CFB41A00EF5004C2E5D204021CF5D20107
:101A9C0080C6D20080C0D20280BCD2D580BAD2051A
:101AAC0080B47F201219F72002077401B54D004055
:101ABC00F11219BCFF1219F7021A30D208D20680A3
:101ACC00951219BCFB1219BCFA1219BCF94A4B70CD
:101ADC000679EC7A1D7BFF20022EE54D602A7E00F4
:101AEC008E8275830012117360060EEE654E70F0D7
:101AFC00C2D5EBC0E0EAC0E0E9C0E0EE121D55D063
:101B0C00E0F9D0E0FAD0E0FB12115AFF60AAEBC06A
:101B1C00E0EAC0E0E9C0E01219F7D0E02401F9D006
:101B2C00E03400FAD0E0FBE54E0460DCD54ED98001
:101B3C0087D20280A2121D3860F7E54E70010412A4
:101B4C000E75A94E600DE54E600914F54E121DDFA1
:101B5C00EF60F3EA30E702F404C3995077EAF42516
:101B6C004E0430E701E404F54E800D121D3860C1BF
:101B7C00EA054E254E120E75EA784BF630E701E475
:101B8C00254E04D54E0420050114121D55E4C0E069
:101B9C00121DDF784BE6601320E70714F61219DFED
:101BAC00802204F6D0E014C0E07F001219DFE54E6D
:101BBC0060071219D6154E800B3005031219D6D0BA
:101BCC00E0021A30D0E00480C5121D3860A0E54E4A
:101BDC0004120E75784BEAF6E54E200502600104FE
:051BEC002404121D5548
:101BF10074FF04C0E0121DDF1219DFE54E2005025B
:101C010060031219D6D0E0B54EE87F451219E97884
:101C11004BE67F2B30E7047F2DF404C0E01219F767
:101C2100D0E075F00A84C0F01219E0D0E01219E09A
:101C3100021A30791080027908C206C2088008D2DF
:101C4100D5790A8004790AC2D5E54E047002F54EB1
:101C5100E4FAFDFEFF1219BCFC7B082001131219E6
:101C6100BCFD7B1030000A1219BCFE1219BCFF7BAF
:101C710020EC3382D592D55013C3E43000069FFF88
:101C8100E49EFEE42001039DFDE49CFCE4CBF8C24C
:101C910001EC700CCFCECDCCE824F8F870F38017AE
:101CA100C3EF33FFEE33FEED33FDEC33FCEB33FBDF
:101CB100994002FB0FD8E9EB300105F8D0E0C448A8
:101CC100B201C0E00AEC4D4E4F78207B0070C2EAB1
:101CD100B54E0040BCC0E0121D57D0F0D0E020014D
:101CE10004C4C0E0C4B201C0F01219E0D0F0D5F0D4
:101CF100EB021A301214051ACD531C34581A9E4C9B
:101D01001A9A421C384F1C40441C40491AB3431CC8
:101D110046551B77461BD5451B41471E0C501AA241
:101D21002D1AA62E1AC92B1AAA231AC7201DF52A65
:101D31001A624800001AC1E54EB4FF03754E06123F
:101D410019BCFC1219BCFD1219BCFE1219BCFF789A
:101D510044020EA4790AA2D5200314300509B91052
:101D6100020404B9080104A2D5200602500104208E
:101D710002689202B54D005034C0E07F2030031953
:101D81007F30A20272067205500F121DAEC202C24E
:101D910006C205C2087F30800F300503E9C0E0129A
:101DA10019F7300503D0E0F9D0E0B54DCC30051777
:101DB1007F30B9100C1219F77F583004077F7880F3
:101DC10003B908031219F73002057F2D0219F77FB5
:101DD100202008F87F2B2006F322920280CF7F007B
:101DE100B4070050052444F8E6FF22286E756C6C98
:101DF1002900D2011219BC3001F8C201784D30D549
:101E01000108F6021A622D504349581219BC2403E5
:101E1100B405004001E4901E07931219E8743A12C8
:0A1E210019E8D203754D04021C34C9
:1021F100E54C30030104F82328243AF822783730DB
:102201000302783AE475F0011213E502115A60EC09
:10221100C5507002154F14C550200304FF02376AE0
:10222100783774FFF5F00213F5FF0236CCE54D6007
:1022310006D54D037F002220030F123702EF6008FD
:102241000550E5507002054F2278371213DC121148
:102251005AFF60E97837E475F0011213E580DE1268
:102261002238EFC0E012222AD0E040F380A0D2034E
:102271008002C2038B378A388939E4F54EF54CF573
:102281004FF550754D00C202C200C201C2041221B5
:10229100FEFF7005AF4E7E0022B425301221FEFFF5
:1022A10024D0B40A00500C75F00AC54DA4254DF593
:1022B1004D80E924CFB41A00EF5002C2E502250C8B
:1022C100D20180D8D20080D4D20480D0EF12222A49
:1022D1005008122260EF600E80A9EFC0E012223890
:1022E100D0E06F609EEF607412220F80A712223837
:1022F100EF6069E54D7007054D8003122238EF60EC
:102301001420040E1221F1E475F0011213E5EF120D
:1023110011A0D54DE6200404054C054E80BA1222C9
:102321002EEFC0E012222AD0E0500412220FE4FF67
:1023310020040E1221F1E475F0011213E5EF1211E0
:10234100A0EF70DA200404054C054E808BE54D604A
:1023510002054D12226012222EEF70C6300304E4F2
:1023610012220FE54E60030222957EFF7FFF22E5D8
:102371004D6002054D122260D206D20512222EEFC7
:1023810030060260D7C0E012220FD0E0AC51AD524E
:10239100AE53AF54122DEA8C518D528E538F54503F
:1023A10007122238C20580D4200410200502054EF0
:0823B1001221F11213DC054CAE
:1023B900121365022284D0E0809A7900800A79108C
:1023C900800679088002790AD205E54D6002054D3B
:1023D900E9C0E0122260EF60DD122238BF2D04D27D
:1023E900028003BF2B09122260EF60CA12222ED08D
:1023F900E0B40A028033B40802802EBF302770028D
:102409007408C205C0E012222ED0E0BF7802800312
:10241900BF5816054DD54D028007D54D04D205800C
:102429000B741080197002740ABF000AEFF8E4FCFB
:10243900FDFEFF0224BFC0E0EF12220FD0E0F9E455
:10244900FCFDFEFFE9C0E0ECC0E0EDC0E0EEC0E05D
:10245900EFC0E012222EEFF8D0E0FFD0E0FED0E08E
:10246900FDD0E0FCD0F0E8604DB461004007B47BDA
:10247900005002C2E524D0503DFA24F6500724F951
:102489005034240AFAEAB5F000502BCFA9F0A42F52
:10249900FF92D5E9C5F0CEA4A2D53EFE92D5E9C5F5
:1024A900F0CDA4A2D53DFD92D5E9C5F0CCA4A2D525
:1024B9003CFCC205808EE8C0E020042A20050805FE
:1024C9004E3002031213101221F11213DC054C20B5
:1024D900000B20010DEE8FF01211D4800912136543
:1024E9008004EF1211A0D0E012220F0222842004EE
:1024F900101221F11213DC054CE54F8550F0121131
:10250900D480E8121405234E5323C75822C54C2200
:10251900C142229D4823CB4F23CF4422EE4323C3FC
:102529004923CF5523704623704523704722C92A72
:0725390024F74E000022CD43
:0D372200ED33EC3360065004EC6480FC22B3
:102EBD00020E6022EDA2E7D2E7F9EC3340F260F3A7
:102ECD00B4FF08ED547F70E8020E6AF82481C2E069
:102EDD00C0E0F40428FAC313FCED92E7FD8C448D99
:102EED00458E468F47EEA2E7E9BA7F02C313340041
:102EFD009400FA75F091A4E5F013F494FE8AF0A411
:102F0D0033E5F033248CD313FDE492E7FE7F007C90
:102F1D003F758302ECC0E0F8EDC0E0F9EEC0E0FAD9
:102F2D00EFC0E0FBAC44AD45AE46AF47120C9BD0B5
:102F3D00E0FBD0E0FAD0E0F9D0E0F8120AA1ED64A0
:102F4D0080FD30E7011CD583CBED33CC33F8D0E0D9
:0A2F5D00A2E71328C313CC13FD22D2
:1030F3008F478E468D458C44AB4BAA4AA949A848B5
:10310300120C9B12299F8F478E468D458C44E548B0
:1031130030E747ECC0E0EDC0E0EEC0E0EFC0E0E434
:10312300FFFEFDFCAB47AA46A945A844120D387B18
:10313300DB600250087A0F7949784080067A0F796C
:103143004978C0D0E0FFD0E0FED0E0FDD0E0FC1233
:103153000AA18F478E468D458C44AF47AE46AD4599
:03316300AC442257
:1026CD003A70FA83BCAAE9E43E81E0F8BF9DE9E6E1
:1026DD003F80000039283C1ABB9969663DA335E35C
:1026ED00BF255DE73FC90FDB418DDBCCC44936EE1D
:1026FD0045C9913FC5B0F83D3F800000C317F53483
:10270D00452FFA73C60AFDDD1227BC04A2E1920023
:10271D001420E0159026CD7404120FA780261227E1
:10272D00BC30E102B20020E0EB8C448D458E468F2B
:10273D00479026E17404120FA7A844A945AA46ABF9
:10274D0047120B92ED4C6007300004EC6480FC22C4
:10275D001227BCC0E08C448D458E468F47902705CF
:10276D007403120FA7A844A945AA46AB47120B92B2
:10277D00ECC544FCEDC545FDEEC546FEEFC547FF76
:10278D009026F57403120FA7D082A844A945AA4636
:10279D00AB47E58230E007120C9BB20080A6EFCB71
:1027AD00FFEECAFEEDC9FDECC8FC120C9B8095ED49
:1027BD0033EC547FCC33920024605007D0E0D0E04E
:1027CD00020E607B837AF97922783E120B92EDF935
:1027DD0033ECF83324815011EFFBEEFA120DF412A5
:1027ED000DB6ECB2E7FC120AA1ED33EC33602F24E9
:1027FD0003F8C313FCED92E7FDE82481E4501FECD0
:10280D00F8EDF9EEFAEFFB120DF4EF04C2E0FCF572
:10281D0082120DC0ECB2E7FC120AA1E58203FAEDBB
:0E282D0033EC3360071413FCED92E7FDEA2252
:100E2B00E9D2E7C933E833F892D5EDD2E7CD33EC0D
:070E3B0033FC5002B2D52286
:100E4200EC30E7100FBF000C0EBE00080DBD000411
:100E52000BEB6014A2D5EB13FCED92E7FD2274FFBD
:100E6200FCFDFEFF22E480F8A2D574FF13FC7D8016
:030E7200E480EF2A
:100E7500F920E72824F950037907E4F42402FB1844
:100E8500DBFDE624FB5014E9600DE4F618E604F6F4
:0F0E9500B40A08E4F6D9F57401F60A22C2D52290
:100EA400ED33EC3392D5FA602AB4FF33EDC2E77B1D
:100EB400FF60067A0E79C9E4227A0E79D220D5042D
:100EC4007A0E79CD224E614E002B494E46002D49B3
:100ED4004E4600E47A08F608DAFC7B00740722E840
:100EE400C0E0ECC0E0EDC0E0EEC0E0EFC0E0EA75C9
:100EF400F010A4CAABF075F04DA42BFBE435F0FC64
:100F0400EA2410FAEB34C5FBEC34D9FCEDC2E7FF5C
:100F140075F056A4F42411C5F0F434C58FF0A42A56
:100F2400E5F03BE43CF620E714121024D0E0FFD0B7
:100F3400E0FED0E0FDD0E0FC120C9B8014F404121F
:100F44001024D0E0FFD0E0FED0E0FDD0E0FC120B96
:100F540092D0E0F8E6FAEDD2E7CD33EC332482FB0D
:100F6400E4C3CF33CFCE33CECD33CD33DBF37B07E6
:100F740075F00A846004F6081B0AE5F0F6088FF0A1
:100F8400740AA4FFACF08EF0740AA42CFEACF050EA
:100F9400010C8DF0740AA42CFDE435F0F608DBDEB8
:030FA400740722AD
:102DD700C207C208C209C20AF9E4F555F556FCFD57
:102DE700FEFFE91006EA20090CB42D04D209D3220C
:102DF700B42B02D32224D0504794095041240A30DF
:102E07000A15F88556F0740AA42872E74051C5F0F0
:102E1700704D85F056D322D208C0E0E4FBFA792042
:102E27007841120B92ECF8EDF9EEFAEFFBD0E0FCEB
:102E3700E4120DC0120AA13007B41555D322240A93
:102E4700200A20B4FE0720071AD207D32224EB60FA
:102E57000424E0700EA2099207D20AC209D322C342
:102E6700020E60E4300A0BE556300902F404A207AB
:102E770092093008EA255520D2E5A2E7920A5002C6
:102E8700F404B4260050D8CCC0E0EDC0E0EEC0E0BA
:102E9700EFC0E0EC121024D0E0FFD0E0FED0E0FD60
:102EA700D0E0FC200A05120B928003120C9B30091C
:062EB70003120DA5C32269
:100FA700C0E0EFFBEEFAEDF9ECF8120B92D0E0F5AA
:100FB700F0EFFBEEFAEDF9ECF812137FA3A3A3A36E
:100FC700E8C0E0E9C0E0EAC0E0EBC0E0C0F0120B27
:100FD7009212138FA3A3A3A3120AA1D0F0D0E0FB10
:0D0FE700D0E0FAD0E0F9D0E0F8D5F0D42247
:10297F00BE1249253E4CCCCDBEAAAAAB3F8000006B
:10298F003E7ADBB03EED63383F24BC7D3F490FDB21
:10299F00ED33ECC2E7CC339200B4FF13ED547F60FC
:1029AF0003020E607FDB7E0F7DC97C3F022A9AC235
:1029BF0001C3947F401E7007EDD2E794904015EF4E
:1029CF00FBEEFAEDF9ECF87F007E007D807C3F1284
:1029DF000C9BD201ED33EC33248430E705E4C0E0E7
:1029EF00806D04FAEDD2E754F0C333DAFD540734A7
:1029FF00002323C0E0CCC0E0F8EDC0E0F9EEC0E06A
:102A0F00FAEFC0E0FBE4120DC0EC24FEFC8C4C8D01
:102A1F004D8E4E8F4F120B927B007A007980783F4C
:102A2F00120AA1ECC54CB2E7FCEDC54DFDEEC54E4B
:102A3F00FEEFC54FFFD0E0FBD0E0FAD0E0F9D0E0D9
:102A4F00F8120AA1A84CA94DAA4EAB4F120C9B8CA1
:102A5F004C8D4D8E4E8F4F90297F7403120FA7A868
:102A6F004CA94DAA4EAB4F120B92D0E0600F248BA6
:102A7F00F582E43429F58312138F120AA130010B6A
:102A8F007BDB7A0F79C978BF120AA1ED33EC336083
:082A9F0006ECA20092E7FC2204
:100FF4003F8000004120000042C80000447A000005
:10100400461C400047C35000497424004B18968086
:101014004CBEBC205A0E1BCA6753C21C749DC5AE7D
:10102400FB60065407601C2323121052EB543860F3
:101034000912103E12104D120B92ECF8EDF9EEFA73
:10104400EFCB22EB12104D80F1543803241C900F87
:10105400F4FE93FC0EEE93FD0EEE930ECE93FF2260
:102F7300022CE7E493A3F8E493A34003F68001F261
:102F830008DFF48029E493A3F85407240CC8C3335F
:102F9300C4540F4420C8834004F456800146F6DF2E
:102FA300E4800B0102040810204080903765E47E22
:102FB300019360BCA3FF543F30E509541FFEE49323
:102FC300A360010ECF54C025E060A840B8E493A3EA
:102FD300FAE493A3F8E493A3C8C582C8CAC583CA15
:102FE300F0A3C8C582C8CAC583CADFE9DEE780BECD
:01376900005F
:10106400E709F608DFFA8046E709F208DFFA803E6E
:1010740088828C83E709F0A3DFFA8032E309F6085B
:10108400DFFA8078E309F208DFFA807088828C83C3
:10109400E309F0A3DFFA806489828A83E0A3F60877
:1010A400DFFA805889828A83E0A3F208DFFA804C51
:1010B40080D280FA80C680D4806980F28033801028
:1010C40080A680EA809A80A880DA80E280CA803391
:1010D40089828A83ECFAE493A3C8C582C8CCC58309
:1010E400CCF0A3C8C582C8CCC583CCDFE9DEE780D9
:1010F4000D89828A83E493A3F608DFF9ECFAA9F058
:10110400EDFB2289828A83ECFAE0A3C8C582C8CCAD
:10111400C583CCF0A3C8C582C8CCC583CCDFEADEC6
:10112400E880DB89828A83E493A3F208DFF980CC28
:1011340088F0EF60010E4E60C388F0ED2402B40421
:101144000050B9F582EB2402B4040050AF232345C8
:0611540082239010B47329
:10115A00BB010689828A83E0225002E722BBFE0293
:09116A00E32289828A83E49322C6
:10117300BB010CE58229F582E5833AF583E0225031
:1011830006E92582F8E622BBFE06E92582F8E2227B
:0D119300E58229F582E5833AF583E4932295
:1011A000BB010689828A83F0225002F722BBFE012E
:0211B000F32228
:1011B200F8BB010DE58229F582E5833AF583E8F073
:1011C200225006E92582C8F622BBFE05E92582C81F
:0211D200F22207
:1011D400BB010A89828A83F0E5F0A3F0225006F766
:0F11E40009A7F01922BBFE06F3E5F009F3192263
:1011F300E88FF0A4CC8BF0A42CFCE98EF0A42CFC9B
:101203008AF0EDA42CFCEA8EF0A4CDA8F08BF0A418
:101213002DCC3825F0FDE98FF0A42CCD35F0FCEB77
:101223008EF0A4FEA9F0EB8FF0A4CFC5F02ECD393C
:0F123300FEE43CFCEAA42DCE35F0FDE43CFC22A9
:1012420075F008758200EF2FFFEE33FECD33CDCC63
:1012520033CCC58233C5829BED9AEC99E5829840E6
:101262000CF582EE9BFEED9AFDEC99FC0FD5F0D6C3
:10127200E4CEFBE4CDFAE4CCF9A88222B800C1B9ED
:101282000059BA002DEC8BF084CFCECDFCE5F0CB2B
:10129200F97818EF2FFFEE33FEED33FDEC33FCEB64
:1012A20033FB10D703994004EB99FB0FD8E5E4F91F
:1012B200FA227818EF2FFFEE33FEED33FDEC33FC0C
:1012C200C933C910D7059BE99A4007EC9BFCE99A00
:1012D200F90FD8E0E4C9FAE4CCFB2275F010EF2F45
:1012E200FFEE33FEED33FDCC33CCC833C810D70745
:1012F2009BEC9AE899400AED9BFDEC9AFCE899F880
:0E1302000FD5F0DAE4CDFBE4CCFAE4C8F92212
:0E131000C3E49FFFE49EFEE49DFDE49CFC22EE
:10131E00EB9FF5F0EA9E42F0E99D42F0EC6480C846
:06132E0064809845F022E6
:10133400EB9FF5F0EA9E42F0E99D42F0E89C45F00F
:011344002286
:10134500BB010789828A830214375005E9F8021424
:101355002BBBFE05E9F802144389828A8302137FB9
:10136500BB010789828A8302139F5005E9F802149D
:0A1375004FBBFE05E9F802145B22ED
:10137F00E493FC740193FD740293FE740393FF22B4
:10138F00E493F8740193F9740293FA740393FB22B4
:0C139F00ECF0A3EDF0A3EEF0A3EFF022C1
:1013AB00A8828583F0D083D0821213C21213C2128B
:1013BB0013C21213C2E473E493A3C583C5F0C583B0
:1013CB00C8C582C8F0A3C583C5F0C583C8C582C88C
:0113DB0022EF
:0913DC00E6FB08E6FA08E6F92236
:1013E500FAE6FB0808E6F925F0F618E6CA3AF62209
:1013F500FAE6FB0808E625F0F9F618E63AFAF622C9
:10140500D083D082F8E4937012740193700DA3A376
:1014150093F8740193F5828883E47374029368608A
:06142500EFA3A3A380DF8A
:1034C900EFB40A07740D1234D4740A309811A8990C
:1034D900B8130CC2983098FDA899C298B811F63063
:0734E90099FDC299F599223B
:1037020010180B123739BF0D027F0A0234C9AF0FEE
:013712002294
:05376A008F0FD21822B0
:1036CC00EFC394094005EF940E4003BF2003D38051
:0336DC0001C32205
:10321C008B2E8A2F89308B348A358936AB2E05302C
:10322C00E530AA2F7002052F14F912115A70ED74A3
:10323C00FF2530F53074FF352FF52FAB310533E515
:10324C0033AA327002053214F912115AFFAB2E0553
:10325C0030E530AA2F7002052F14F9EF1211A0706F
:08326C00DAAB34AA35A93622C1
:10000E00E4FFFE12115A600C0FEF70010E09E97039
:05001E00F20A80EF2250
:0C142B00E6FC08E6FD08E6FE08E6FF22ED
:0C143700E0FCA3E0FDA3E0FEA3E0FF2228
:0C144300E2FC08E2FD08E2FE08E2FF22E5
:0C144F00ECF608EDF608EEF608EFF622C9
:0C145B00ECF208EDF208EEF208EFF222CD
:0A3739003098FDAF99C2987E00227F
:00000001FF
